S00D000074696D65722E73726563F6
S113000012C02BC02AC068C128C027C026C025C082
S113001024C023C022C021C020C01FC01EC01DC0D8
S11300201CC01BC01AC011241FBECFE5D4E0DEBF24
S1130030CDBF10E0A0E6B0E0E0E5F9E002C0059035
S11300400D92A437B107D9F710E0A4E7B0E001C0DE
S11300501D92A339B107E1F736C4D2CFCF93DF9312
S1130060CDB7DEB722970FB6F894DEBF0FBECDBF73
S113007080918100909182002CE330E0B90154D446
S1130080CB018093770080918100909182002CE3D2
S113009030E0B90149D489839A8389819A812AE01D
S11300A030E0B90141D4CB018093780089819A81F1
S11300B02AE030E0B90138D489839A838981809316
S11300C0790022960FB6F894DEBF0FBECDBFDF9144
S11300D0CF910895CF93DF93CDB7DEB7909177009A
S11300E08CE3989F90011124909178008AE0989F66
S11300F0C0011124280F391F809179009927820F9C
S1130100931F9093820080938100DF91CF91089593
S1130110CF93DF93CDB7DEB721970FB6F894DEBF48
S11301200FBECDBF898380913C0099278270907067
S11301300097C9F78981282F3327C901820F931F9C
S1130140D4D3909382008093810088DF21960FB6E8
S1130150F894DEBF0FBECDBFDF91CF910895CF934A
S1130160DF93CDB7DEB721970FB6F894DEBF0FBE8D
S1130170CDBF898380913C0099278270907000974D
S1130180C9F78981282F3327C901820F931F6091F2
S1130190810070918200B6D380913C0099278270CF
S11301A090700097C9F721960FB6F894DEBF0FBE82
S11301B0CDBFDF91CF910895CF93DF93CDB7DEB755
S11301C021970FB6F894DEBF0FBECDBF1982898187
S11301D08F3F09F405C0000089818F5F8983F7CFC1
S11301E021960FB6F894DEBF0FBECDBFDF91CF913D
S11301F00895CF93DF93CDB7DEB722970FB6F89467
S1130200DEBF0FBECDBF19821A8289819A812BE08D
S1130210883B920708F007C0CFDF89819A81019655
S113022089839A83F2CF22960FB6F894DEBF0FBE6D
S1130230CDBFDF91CF910895CF93DF93CDB7DEB7D4
S113024010922B0010922A0080E8809340008FEFD8
S1130250809337008FEF809334008FEF80933100C9
S11302608FEF809338008FED809335008FEF80936C
S1130270320010927B0082E080937C0010927D001B
S113028010927E0010927F0080E042DF1092800086
S113029010927400109275001092760083E080939F
S11302A07300DF91CF910895CF93DF93CDB7DEB77D
S11302B088E08093420087E08093450010924400D8
S11302C080E28093430080915900806880935900B4
S11302D07894DF91CF9108951F920F920FB60F92E9
S11302E011242F933F934F935F936F937F938F9337
S11302F09F93AF93BF93EF93FF93CF93DF93CDB7C8
S1130300DEB71092440080918100909182000197A1
S11303109093820080938100A1DE8091810090916E
S113032082000097B1F481E0809380001092750000
S11303301092740083E080937300109259008BE054
S1130340809377008CE0809378008DE0809379002F
S11303507894DF91CF91FF91EF91BF91AF919F91ED
S11303608F917F916F915F914F913F912F910F905A
S11303700FBE0F901F901895CF93DF93CDB7DEB7C4
S113038021970FB6F894DEBF0FBECDBF8FEF8093D9
S113039037008FEF809334008FEF809331008FEF1D
S11303A080933800809173008C6D809335008FEFBB
S11303B08093320080917B008F5F80937B008091DB
S11303C07B00843010F010927B0080917B00992791
S11303D0FC01E159FF4F908180917300892B809338
S11303E0350080917B008330B1F5809175008823BE
S11303F039F080917400882319F088E089830FC054
S113040080917500882319F080E2898308C0809167
S11304107400882319F081E0898301C019828091D6
S11304207600882321F48981846089830FC08091B8
S11304307600813021F489818260898307C08091AC
S11304407600823019F4898180618983898180955D
S11304508093320054C080917F00882371F1909181
S11304607B0080917C00981741F580917D008F5F1F
S113047080937D0080917D00893C60F080917E00B6
S1130480813019F410927E0003C081E080937E00D5
S113049010927D0080917E00813079F480917B0000
S11304A0882329F480916A008093320028C08091C7
S11304B06A0080688093320022C080917B00882388
S11304C079F480917B009927FC01E958FF4F8081E2
S11304D09927FC01E05AFF4F8081809332000FC0BE
S11304E080917B009927FC01E958FF4F808199276F
S11304F0FC01E05AFF4F808180688093320021968E
S11305000FB6F894DEBF0FBECDBFDF91CF91089533
S1130510CF93DF93CDB7DEB722970FB6F894DEBF43
S11305200FBECDBF109231008FEF809332008091C7
S113053073008C6F809335008EEF809338003CDE1F
S113054080913000809589838981882361F11A82A2
S11305508A81883008F045C08981282F33278A8111
S1130560992702C0359527958A95E2F7C9018170CC
S11305709070009771F08A819927DC01A557BF4FCD
S11305808A819927FC01E557FF4F80818F5F8C9307
S113059006C08A819927FC01E557FF4F10828A81A2
S11305A08F5F8A83D5CF1A828A81883008F019C078
S11305B08A819927FC01E557FF4F8081823068F0DA
S11305C08A819927FC01ED57FF4F81E080838A815E
S11305D09927FC01E557FF4F10828A818F5F8A8338
S11305E0E3CF22960FB6F894DEBF0FBECDBFDF91E6
S11305F0CF910895CF93DF93CDB7DEB722970FB68F
S1130600F894DEBF0FBECDBF80918000882319F11E
S11306101A8219828981883008F013C08981992748
S1130620FC01ED57FF4F9A818081890F8A8389816C
S11306309927FC01ED57FF4F108289818F5F8983D1
S1130640E9CF8A81882309F435C110928000809112
S113065076005EDD2FC180917400882329F4809197
S11306607500882309F40FC019828981883008F045
S113067021C189819927FC01ED57FF4F108289819F
S11306808F5F8983F2CF809185008823A1F019823E
S11306908981883008F00AC089819927FC01ED57C7
S11306A0FF4F108289818F5F8983F2CF1092760089
S11306B0809176002DDD809184008823A9F0198231
S11306C08981883008F00AC089819927FC01ED5797
S11306D0FF4F108289818F5F8983F2CF81E08093FD
S11306E076008091760014DD809187008823A9F03C
S11306F019828981883008F00AC089819927FC0110
S1130700ED57FF4F108289818F5F8983F2CF82E09A
S11307108093760080917600FBDC809183008823AF
S1130720D9F019828981883008F00AC08981992713
S1130730FC01ED57FF4F108289818F5F8983F2CFCF
S113074081E08093740082E08093730010927F00B4
S11307508091760004DDA8DD809186008823E9F08D
S113076019828981883008F00AC089819927FC019F
S1130770ED57FF4F108289818F5F8983F2CF81E02B
S11307808093740081E0809375001092730010923E
S11307907F0080917600E3DC87DD809188008823E8
S11307A0D9F019828981883008F00AC08981992793
S11307B0FC01ED57FF4F108289818F5F8983F2CF4F
S11307C081E08093750081E08093730010927F0034
S11307D080917600C4DC68DD80918900882309F467
S11307E048C019828981883008F00AC08981992714
S11307F0FC01ED57FF4F108289818F5F8983F2CF0F
S113080080917F008823A9F180917C009927DC01E5
S1130810A958BF4F80917C009927FC01E958FF4FEC
S113082080818F5F8C9380917C00813089F48091EA
S11308307C009927FC01E958FF4F80818630C0F085
S113084080917C009927FC01E958FF4F108210C069
S113085080917C009927FC01E958FF4F80818A3000
S113086038F080917C009927FC01E958FF4F1082F1
S113087031DC80918A008823E9F0198289818830EB
S113088008F00AC089819927FC01ED57FF4F1082B7
S113089089818F5F8983F2CF80917C008F5F809301
S11308A07C0081E080937F0080917C00833010F095
S11308B010927C0022960FB6F894DEBF0FBECDBF17
S11308C0DF91CF910895CEE5D4E0DEBFCDBFB4DC97
S11308D01FDE90DE198289818F3008F0F9CF4CDD5C
S11308E06BDC89818F5F8983F6CFE199FECF9FBB53
S11308F08EBBE09A01960DB29FBB8EBBE09A802D11
S11309009DB30895FFEF0FB6E199FECF9FBB8EBB59
S11309106DBBF894E29AE19A0FBEF0FF08958F5FE1
S11309209F4F672FFF27F0CFAA1BBB1B51E107C0C6
S1130930AA1FBB1FA617B70710F0A61BB70B881F6B
S1130940991F5A95A9F780959095BC01CD010895FA
S113095040792430191202780010772F21117FF882
S1070960F4ECDC03D0
S9030000FC
